:020000040000FA
:100000003F3F3F3F20067E213C7E296B0F86FFB796
:100010000115CECCCCFF0800FF0802FF080486AA19
:10002000CE00001653A700E701A100260DE101262E
:100030000908088C000E26ED20078699B7080220D3
:10004000DD815527034320D88E000DDE0FFF080801
:10005000DE11FF080A8601B70812CE0100A600A72C
:1000600000088C011026F6BD600B86FFB7011686CE
:10007000009797B70813B70814B70815B701D3B797
:100080000157B70624B70142BD252E8E07FF860112
:10009000B718018600B7180097CFBD2344BD27CC01
:1000A0007F001A86019700BD61AEBD6172DED94343
:1000B000A100261853E101261396004C810A26E57B
:1000C000BD26269697819227037E20F6C663F70108
:1000D000608601971ABD611C96978192260A961A2E
:1000E0004C810A26EEBD26D88601971ABD60CE96B1
:1000F0001A4C810A26F47F0C097F0C087F0C0B86B2
:10010000F0B70C0A862DB70C09860FB70C0BB60C8E
:1001100008B60C0A7F015FBD2A9B7D001A27058661
:1001200095BD52D57D001927058696BD52D57F0015
:10013000197F001A0E3E0FBD235720F80FCE214E17
:10014000F60C20C40EBD4C24AD00BD23573B215EF0
:100150002B1A216622EA522E5EBB22422242B60CA4
:1001600020840E27F939BD34C5B60C08F601ECC160
:10017000FF270AC5102706168A807E218BB7013615
:10018000815C2706BD52C9B6013616F70136B701A4
:1001900037813024068651BD52D5394D2A05847FDA
:1001A0007E225381392204BD399C39CE2142165812
:1001B000BD4C24AD00393BFE4CB53C164C664D356C
:1001C000224235F93C0F43DE43E344DD3A9639548D
:1001D0003A3159D55DE322425D1659FB5A1B5D2623
:1001E00053AB3BE83BF35C663BDF3BD85C9A60BEBD
:1001F00060C359495C365C1D5ABC529F5C4D22431A
:100200005C045B475B185AE9596A59975B775BA6B0
:100210005BD54D103C083AB43A70224222423A83F0
:10022000239744F644F061C261C743DE43E34D10B7
:100230002397224222422242224222422242224248
:10024000224239BD26D8860136BD60CE324C810AA5
:1002500026F639CE2268A10027090808088C22B0AA
:1002600026F439EE01AD00393146E73246EB33462C
:10027000EF3446F33546F74035F95346C75446CB7D
:100280005046CF5146D33A46D73C46E36946DB4118
:1002900046DF5F5C04595C365A5C1D7261C2736153
:1002A000C77443DE7543E3764D107723975C529F06
:1002B000F71802B71803DFCD96CF8A01B718018669
:1002C000D2B7180039F71804B71805DFD086D2B7AF
:1002D000180197CF39F71806B71807DFD396CF84E0
:1002E000FEB7180186D2B7180039B6180197CC8529
:1002F000012709BD2315DECDAD0096CC8502270967
:10030000BD2326DED0AD0096CC85042707BD233360
:10031000DED3AD003996CF8A01B718017F1800B639
:100320001801B61802397F18017F00CFB61801B640
:1003300018043996CF84FEB718017F1800B618014B
:10034000B6180639BD2326BD2315BD2333CE23564B
:10035000DFCDDFD0DFD339F60624271AC1102507F9
:100360008677BD52D5200958CE2377BD4C24AD00E9
:100370007F0624BD292D39237623762A085292231D
:1003800076237623762A70237623762A762A7F238D
:1003900076237623762376F60124B601258101277C
:1003A0001081022633B601235D27058B0A5A26FBEE
:1003B00016C11E250FF701248673C601CE0124BD88
:1003C00028E2200DC110241058CE23DFBD4C24ADEF
:1003D00000BD3932BD471F398628BD52D520F223D2
:1003E000D7247E23FF5431542B255D256825CE4329
:1003F000884392439C25D423D723D723D723D7BD23
:10040000254C8D0C960527058697BD52D57E246E0A
:10041000CE4000DF00CE20004F8D36C601112702EE
:100420008D3ACE6000DF00CE40004F8D24C6021111
:1004300027028D28CE7FC0DF00CE60004F8D12CE08
:100440008000DF00CE7FE08D08C6031127028D0CEF
:1004500039AB0089000C089C0026F6399705260365
:10046000730005F708008697B708028D06398D03DB
:100470008D013986D008095A26FB4A26F839BD2550
:100480004C8D0C960527058698BD52D57E246E9618
:10049000868A809786B70812CE000C860C9706864F
:1004A0000197004C9701A60097028601A7007300F0
:1004B00000730000A100262C482504A70020ED961B
:1004C00002A700088C0800275B7C000626D896034C
:1004D00084809703970496008B021997008B01196B
:1004E000970120C2850F261FE600C4F01127C99787
:1004F00005960426CA96017C0004B708008698B7C2
:100500000802BD247320B8E600C40F1127AA97057E
:100510008698B7080296007C0003B70800BD2473D4
:10052000861020889686847F9786B7081239B60889
:1005300016850427164F970397049705BD248FBD92
:100540002410960597192703BD246E39BD49434FE2
:1005500097037F080097049705392001E5B6064305
:100560008AFFB706437E2A12868097459744BD448A
:10057000FCCE0000DF2FDF33DF3BDF3DDF3F8601B6
:100580009740CE0002DF31CE6006DF358601BD60C8
:10059000CE8601972FCE6006DF31CE3012DF358652
:1005A00002BD60CECE3012DF31CE6018DF3586035B
:1005B000BD60CEF60816C520270FCE6018DF31CEFD
:1005C0000026DF358604BD60CE86017E611CBD5DE0
:1005D000EA7E5F92BD4943B608165F85102602C6C3
:1005E0001085082602CA01F708045F85202602C686
:1005F0001085042602CA01F708035F85402602C65B
:100600001085022602CA01F708025F85802602C60D
:100610001085012602CA01F70801BD2473BD2473A9
:10062000BD24737E2473CE0047BD42DA16263FCE2A
:10063000004BBD42DA162636CE004FBD42DA1626F2
:100640002DCE0053BD42DA162624CE0057BD42DA25
:1006500016261BCE0027BD42DA162612CE002FBD6D
:1006600042DA162609CE0033BD42DA162708BD2627
:10067000D886927E52D59662F60816C50127048167
:100680000B200281022AE74FBD52D5CE0100A60001
:10069000A700088C011626F6BD600B7F0643B60145
:1006A00001847FB701017F008196188A409718BDA9
:1006B0003932BD2932BD539FBD5D7EBD64829645F2
:1006C00026037E4C662A037E4D35810126037E4C2F
:1006D000B5810226997E4D10CE001B4FA700088CD5
:1006E000011126F8B7014297179718B70812B701FA
:1006F00046B701478601B701018602B70645C69095
:10070000F7010FBD600BBD2A88CEFFFFFF0111FF6F
:100710000113FF0115BD2B11BD23448603979AB722
:10072000013EC602F7013F86FF9765CE0003DF0456
:10073000DF1DDF21DF298610972CF60816C501275B
:10074000048608200286019762BD5D7EBD27C4270E
:1007500008B601018A08B70101BD5949BD59D5BD87
:100760005ABCBD5C04BD5C4D861EB70108867FB7D0
:100770000109CE0003FF080ABD5E14B6011184F71B
:10078000B7011186019740974386049736860297F2
:1007900032973A8603974A8606974E86099752867D
:1007A0001297568615975ABD61D2861497468620B1
:1007B00097608620978BBD44FCB601EA2603BD30C6
:1007C000317E26A936B6081685103239BD28AFBD50
:1007D0002A887F06388DED270F7F0639730639B6D4
:1007E00001018A08B7010139B77FC1B77FC0B77F60
:1007F000C386FFB77FC2863CB77FC3B77FC186245D
:10080000B77FC3B77FC18601B70624CE0805FF06B0
:1008100025CE0064FF0627BD28447D7FC2C61FF792
:100820007FC27D7FC12AF0F17FC026EB86FFB7062D
:1008300039BD29A7B70649BD29A7B70648BD292D47
:100840007E29A139FE062709FF06278C000026090C
:10085000BD285ACE0B00FF062739B601158A03B70B
:100860000115CE080086FFA700088C080626F8FEB2
:1008700006258C08002607F60624C5012724F6065F
:1008800024C803F70624C501270409FF0625FE0630
:1008900025F60624B6011584FC1BB7011586FFA7B3
:1008A0000039CE0805FF06258602B7062420DF4F53
:1008B000CE061CA700088C062426F8BD27C42708EE
:1008C000CE9501FF061E2006CE0100FF061EB608CB
:1008D0001685202605CE60182003CE5026FF06225E
:1008E000395FBD27C4270139FF063E7F063A7F06E0
:1008F0003B7D06392605BD2A4C20F67F06398D162C
:10090000178D135D270FFE063EA60009FF063E8DDC
:1009100005095A26F1397F063A7F063B7D7FC32BB6
:1009200005BD2A4C20F67D7FC2B77FC23986418D36
:10093000E539BD27C42701397F063A7F063B7D068E
:10094000392605BD2A4C20F67F063986638DC78679
:10095000088DC3C606CE0111A6008DBA085A26F826
:10096000B601018DB1B601088DAC39B67FC12B0639
:100970008680BD52D53B8D013B8624B77FC18D2734
:1009800027392B3E811E26037E208BB706248D1728
:10099000B70625270C16CE06268D0CA700085A266A
:1009A000F88625B77FC1397F063A7F063BB67FC1FF
:1009B0002B05BD2A4C20F6B67FC03986FFB7063915
:1009C00020DF432739F60101C5082709F6064485CB
:1009D00001271E2012F60644CA0185012713CA0208
:1009E0007D06452602CA8085022704CA042002C467
:1009F000FBF706447D064527037A064520BDF6062B
:100A000038CA80F706382099BD52C9B60101850859
:100A1000261E7D00172A0A7D0643260586037E5280
:100A2000D5B601018A08B7010186538D157E4CA702
:100A3000B6010184F7B701018602B706457F064378
:100A40008654BD28E1BD5CF3BD5478393637FF06C6
:100A50003CB60816850827127A063A260D86FFB797
:100A6000063A7A063B26037E208B3332FE063C395B
:100A7000B606267E52D5B606388A01B7063839B68C
:100A8000063884F0B70638394FF60639CE0624A763
:100A900000088C064726F8F70639398D128D2AB6DC
:100AA00001EA2705BD30E02003BD30317E2B1ACE90
:100AB00001434FA700088C015E26F8CE0165FF01B7
:100AC0006197DCB70C137E338CBD36F4BD35C47F23
:100AD00001ED7F01EC7F015F8602B70C1586ABB795
:100AE0000C11860BB70C12860AB70C178622B70CAE
:100AF000158684B70C1586BDB70C15B601608A80C3
:100B0000B70160BD36507F0C158620B701557E3584
:100B10001FBD35CEBD35A97E3580B60C12F60C1141
:100B2000B701ECF701ED8502270CBD35CEBD2BB822
:100B3000B601ECF601ED8501270CBD35A9BD2BB83A
:100B4000F601EDB601EC8508270CBD2BB8BD354B81
:100B5000B601ECF601EDC5022709BD2BBCB601ECD0
:100B6000F601EDC50127037E314BC5202709BD2BBA
:100B7000B8BD2BB27E3294C5082709BD2BB8BD2B5A
:100B8000B27E3715C580272FB60C15847F810526C8
:100B900007C680F7015F201A8160250AF6015F2AE7
:100BA00011B70C15200CBD2BB8811526058670B722
:100BB0000C15860FB70C15397F015F39FE014B26E6
:100BC00015FE014DAD00FE014B260B7D00DB27011C
:100BD0003986237E52D5AD00FE014B2605C606F7A9
:100BE0000C15B70C10B601ED84FDB701EDFE014BFD
:100BF0002617FE014F8C2D062607865CBD35ED209D
:100C0000088C30B32603BD30B439FE0151A6004430
:100C10004444448A30CE2C1CFF014B39FE0151A6BE
:100C200000840F8A302005FE0151A60009FF015102
:100C30007C0149F60149FE014FE100270F5D2B07BA
:100C4000CE2C27FF014B39CE2C0A20F7FE014F088E
:100C50000808FF014FE600260C7F014B7F014C394D
:100C6000FE014FE600C480F70149EE01FF01515D2E
:100C70002B07CE2C27FF014B39CE2C0A20F78656A6
:100C8000BD35ED8639BD35EDCE2C97FF014FCE2C0D
:100C90007EFF014D7E2C60022C9F5E05720041405C
:100CA000CE2CAFFF014FCE2CA0FF014D7E2C600259
:100CB0002CF004001202007D0100860108170101DA
:100CC000000101010101020101030101040101050B
:100CD00001010601010701010801010901010A01E1
:100CE000010B01010C01010D01010E01010F003981
:100CF00040CE2D00FF014FCE2CF1FF014D7E2C6028
:100D000081009701306B00D643C1112502203B586A
:100D1000CE2D24BD4C24AD00FF014FCE2D07FF0189
:100D20004D7E2C602D462D542D742D942DB42DD434
:100D30002DF42E232E362E362E462E542E622E7055
:100D40002E7E2EEF2F3C8623200286537F014B31CF
:100D5000317E52D57D01472610CE2D5D39022D689A
:100D600084002A063070004643CE2D6D3984002A57
:100D7000043074007D01472610CE2D7D39022D8868
:100D800084002E063070004946CE2D8D3984002E09
:100D9000043074007D01472610CE2D9D39022DA808
:100DA000840613063070004146CE2DAD39840613FB
:100DB000043074007D01472610CE2DBD39022DC8A8
:100DC000840617063070004246CE2DCD39840617B2
:100DD000043074007D01472610CE2DDD39022DE848
:100DE00084061B063070005346CE2DED3984061B59
:100DF000043074007D01472604CE2E0839CE2E0122
:100E00003982007701306B00022E1F840075053097
:100E10007001302F022E1F820077032E22005053C4
:100E20000A5353CE2E2739022E32820061032E350B
:100E30000057440A534DCE2E3A39022E4584004ABB
:100E4000063070004B4DCE2E4A39022E4584004E9E
:100E500006307000CE2E5839022E458400520630DE
:100E60007000CE2E6639022E458400560630700082
:100E7000CE2E7439022E4584005A06307000BD2FE4
:100E8000B1CE2FEDFF01E19662CE01D8BD4C4C7F73
:100E900001D79663CE01D4BD4C4CCE01D7DFC1CE75
:100EA00001D4DFC3DFC5860297C7BD4992B601D51D
:100EB000270F81012621B601D48131241A20023066
:100EC00001CE2EBFDFC1CE01D4DFC5DFC3860297BE
:100ED000C7BD49AF7E2F55CE01D4DFC1DFC5CE2EB1
:100EE000BFDFC3860297C7BD49AFCE01DF207BBD00
:100EF0002FB1CE2FE9FF01E1966227204A2730CE9D
:100F000001D4BD4C4CC603F701E3C62DF701DF8ABF
:100F100030B701DE8630B701DD7E2FDC8602B701F7
:100F2000E38631B701DF8630B701DECE01E03986D6
:100F300001B701E38630B701DF7E2FDCBD2FB1CED4
:100F40002FEBFF01E19663811F2414801E434CCEDA
:100F500001D4BD4C4CC603F701E3CE01DF20158060
:100F60001ECE01D4BD4C4CCE01DFC62DE70009C614
:100F700004F701E3B601D5271B84F0270C44444451
:100F8000448A30A700097C01E37C01E3B601D58ADD
:100F900030A70009B601D4444444448A30A700096C
:100FA000862EA70009B601D4840F8A30A7007E2FB1
:100FB000DC8602B701E0CE01DFFF01E47F01E97DBD
:100FC0000147260C8603B701E6CE2FF0FF01E73973
:100FD0008601B701E6CE306BFF01E739CE01E07D37
:100FE000014727030808083941524556454C0A4D28
:100FF00044CE3000FF014FCE2FF1FF014D7E2C601B
:1010000084061701307400CE3016FF014FCE300732
:10101000FF014D7E2C6084061303307001302F8455
:10102000002A03307001302F82006101306B002CE8
:10103000207D0C142A0139DE23FF01D4DE25FF01B7
:10104000D6CE3031FF014DCE30587D01472703CE3B
:101050003064FF014F7E2C600230638401D706307C
:10106000700052468401D7043074000A5A48303068
:10107000300A303030CE3084FF014FCE3075FF0162
:101080004D7E2C6003308A000A4D4FCE309AFF010E
:101090004FCE308BFF014D7E2C6001015700CE30CA
:1010A000ADFF014FCE309EFF014D7E2C60010C1331
:1010B00001015500BD354BB60155845AB70155B7EE
:1010C0000156B70158BD34EB20D4B70145CE30DC12
:1010D000FF014FCE3031FF014D7E2C6001014500F4
:1010E000CE30E9FF014F7E312E0230F60230F4019E
:1010F000306B0038573340CE3100FF014F7E312E28
:1011000002310801306B005553CE3112FF014F7E82
:10111000312E02311A01306B004453CE3147FF01AA
:101120004DCE312AFF014F7E2C6001306B00CE3155
:1011300047FF014D86FFB700DCBD2C60F601EDC511
:101140000227037E2BBC397F00DC398681B70C1562
:101150007F014AB60C10814027237D015D2B25FEBF
:101160000161A70008FF0161810A270CF60C14C574
:10117000202605BC016326037E31B22020C6FFF77E
:10118000015D20DB7F015DFE0161A70008FF0161B9
:1011900020E6F6014A2A1A7F014ABD319DF6014A2E
:1011A000260FC603F70C15C684F70C15C677F70192
:1011B0004A39FE01618C016526037E319DCE0165B1
:1011C000A60008FF01EF7D01462649BD37224D27C5
:1011D000327D01432A037E329A81C22605BD311B2E
:1011E000201B81C427102408814227048143260D37
:1011F000D645C1822607C680F7014A2003BD319D2E
:10120000BD32A3FE01EFBC016126B5CE0165FF0131
:10121000617E319DF60146C120240F36CE3231BDAC
:101220004C247F014632AD0020D98625BD52D52001
:10123000D2322A3249325233CB32533257326132B0
:10124000743278327F325230CA813126058604B733
:10125000014639B70147391686425D2A014C7E2185
:101260008B813027098131270886207E52D57E5D0B
:10127000EA7E5E14B7015739368669BD35ED328195
:1012800030250C813A2408C612F701467E35ED86DA
:101290006A7E35EDB60144260A39B701447F014321
:1012A0007E3203162B0B813025037E35EDB70146C8
:1012B0003981E9240916CE3243BD4C246E008620C4
:1012C0007E52D532BE32BE309E2CF1337F32942C0A
:1012D0007E33442FF13385338C33D330312CA053FC
:1012E000B253CF5DEA5E1433913AA93C2A3C343CB8
:1012F0003E3C48339261EA3393339D33A733B13395
:10130000BB4D644D6B4D754D7A332D333953F833E6
:10131000C533C82D0732BE37182D07300730753357
:10132000CB3594308B2A302A12496A49719645810F
:1013300082260586427E35F5399645818226F986D4
:10134000437E35F5CE0572C65EBD33568657BD3534
:10135000ED86397E35EDF7015E7D0C162AFBB60C65
:1013600012F60C11C5012607C5EA27ED7E2B20B623
:101370000C10A700BD319D09F6015E5A26D83986AA
:10138000FFB7014339CE01C6FF016339CE016620A4
:10139000F73939863CBD35ED86317E35ED863CBD6D
:1013A00035ED86327E35ED863CBD35ED86337E35B6
:1013B000ED863CBD35ED86347E35ED863CBD35EDA4
:1013C00086357E35ED7E45057E44FCBD4D64863E0A
:1013D0007E35ED8600B70111B70112B7011386F013
:1013E000B70114869FB70115CEDDDDFF0800FF08A9
:1013F00002FF0804FF08057F00CFCE0012C604BD1F
:101400003356DE0FFF0808DE11FF080ACE0811C6AA
:1014100002BD3356CE0086C601BD33569686B70848
:1014200012CE0813C601BD3356CE0100C601BD332E
:1014300056CE0101C601BD3356CE0102C601BD33F1
:1014400056CE0103C601BD3356CE0104C601BD33DD
:1014500056CE0105C601BD3356CE0106C601BD33C9
:1014600056CE0107C601BD3356CE0108C601BD33B5
:1014700056CE0109C601BD3356CE010AC601BD33A1
:1014800056CE010BC601BD3356CE010CC601BD338D
:1014900056CE010DC601BD3356CE010EC601BD3379
:1014A00056CE010FC601BD3356BD600B394D260126
:1014B000398150250BB601558A01B701557E351F7C
:1014C00086207E35358601F60116C5082601397E4F
:1014D0003535860220F186107E353586807E35359D
:1014E0007D01D327013986087E3535B601105F8529
:1014F000012702CA1085022702CA4085042702CAB2
:101500000285082702CA0817BA0155B7015553F4D6
:10151000015653F40155F70155F40156F70156B63B
:101520000155B101582601398604B50C132605B5BD
:101530000154270139BA0154B70154B60C13854040
:10154000270139BA0154B7015420037F0C13C60197
:10155000B60154B5015727048A40C609F70C15B7E0
:101560000C13B10C132716F60116C501260F7F0CBC
:1015700013B7015439B60154854026B9397F015457
:10158000B60C13F6011685402704C4FE2002CA01DA
:10159000F70116394FB70C13B70154B70155B7010E
:1015A00056B70158BD34EB20D7F60116CA06B60C63
:1015B00014858226088544270BC4FB2002C4FDF74E
:1015C000011620B1B601168A06B7011620A7B6018A
:1015D000EC851026037E36F4B6011684F7B70116A3
:1015E000B6010A8A01B7010A86517E28E1F601ECAC
:1015F000C5102601395F7E218BF601372B40968876
:101600002731F60125C101270BC102270C8622BD17
:1016100052D5201FB60124200DB60123F601242740
:10162000058B0A5A26FBBD36B65D27E1C1FF2706AA
:10163000B70160BD36507F0088BD3932200D860D60
:10164000B70C158605B70C15BD35CE860F7E46FB4B
:10165000B6080F85202649858026088540260884FF
:101660001F20068632200286288D4B5D2707B70192
:1016700060C1FF260139C1012702861F841FF70CB4
:1016800014B70C1686E0B70C167F0C15C580270A18
:1016900086FFB701EABD311B20037F01EA7E35A931
:1016A000B60160847F8D0F5D26C18695BD52D5B68B
:1016B000080F84DF20A1813C241C8132241A812858
:1016C0002420811F24107D01602B08F60C16C41FF6
:1016D000112719C601395F398632C680F50C142BE3
:1016E0000B398628C640F50C142601397D01602B84
:1016F00002C6FF39B601168A08B70116B6010A8478
:10170000FEB7010A8652BD28E1BD39327D0043266D
:10171000037C004339BD2AAF8657BD35F586307E40
:1017200035F5847F8140243481302441812B260A81
:10173000B601592A037E37C14F39812D2618B601CB
:10174000592B7E7D011927078680B70119206F86E6
:10175000FFB7015C4F39812E270F206284DF815B48
:10176000245CF601592A2A20488647205A813A24C7
:101770004DF601592A022039D688C4FC27497F003A
:1017800088C51027398130260486A0203A86A220F9
:10179000368145260C7D012527278640B701192073
:1017A0001DB7015A8D25E600271786FFB701594F4F
:1017B000398D18E600270A11270B080820F54F205D
:1017C0000686802002A6017F015939CE3756F601E0
:1017D0005A58BD4C2439380C38173828383138401D
:1017E000385C385D386C386F3872387738783883C1
:1017F000388A389F38AC38BF38CB38CC38E538FA1F
:1018000039053908390A391F392C3931418E310EE1
:101810003292339439960030584F583158326333EE
:101820006450A84C0253060059E443A430E231E46A
:1018300000465353DE548857533148324C334D00E1
:1018400042AE463A4DAE4E435741305B4F5B315B43
:101850003262336134603565366637670052534E05
:10186000544954315441504251533A005A6B005A32
:10187000A600464250D400005A45309C4F9C319EF1
:1018800032CA00318C329A45A8005A6E47865345B9
:1018900030B24FB231B432B633B834BA35BC00309E
:1018A000CC4FCC31CE410849CE4DE20041D64290DA
:1018B00043D84B984C8C4DDA50D052E05384004CB6
:1018C000A8305D4F5D315D325233550043574C5760
:1018D00031A230A04FA0420A4D0E460C41AA444E00
:1018E000554B53DC0046694D3E536A506954564E81
:1018F00010571455C644C8566F00315F3259335AD9
:101900004916528A0050420045AC3468313D323BA2
:10191000333E303D4F3D35BE36C037C238C400314E
:10192000B432B633B834BA35BC30B20030E631E840
:101930000000CE0124FF0128FF012ECE01175FE732
:1019400000088C012626F8D793D79AF70092F70162
:1019500040D78839D69A27037E3932FE01288C0178
:10196000242608F60125C580260139F60125C58003
:101970002709C47FF10140271420045AF7012508E4
:101980006F00FF0128BD45F77A01402006F70125C9
:10199000BD468DF6012526037E471F39840FD68864
:1019A000270EC50127037E60CEC50227FC7E611C81
:1019B000D64326037E5356C10826148100270D8185
:1019C0000522091B9743BD62327E3C1D7E5356D6CD
:1019D0009A2703BD39327D01192632F60125260EDC
:1019E000BD450E4D2608F60116C508260139FE0133
:1019F000288C01192F16A700F60125C5802B037C22
:101A0000012509FF0128BD45427C014039F6011935
:101A1000C40F2606CE0118FF0128FE01288C0116EE
:101A20002F0AA7007C011909FF01283986027E537D
:101A300056D688C50227087F008886107E46FBD6CA
:101A40009A2703BD3932F601252603BD450EF6005F
:101A500093C102270E7C0093BD4542B601258A80C2
:101A6000B70125398640B70119CE0118FF01283981
:101A7000D69A27037E3C20964381072750C60486CA
:101A8000022055D69A27037E3C2096438107273DA6
:101A9000C60386052042D69A27037E3C20964381C2
:101AA00007272AC6028608202FD69A270139C601A1
:101AB000860B2024D69A27037E3C20964381062756
:101AC0000C810727082BA9BD39327E61EA8604C63E
:101AD000067E3AD8860AC601D79A36F60125C40F83
:101AE000F70125B60119275E85022605B6011820E3
:101AF0000DB60117F6011827058B0A5A20F9B70110
:101B00001781102509328603BD53567E3932B6013E
:101B100025F601192B05BB011720227D0117271D72
:101B20004D27064A7A011720F2CE011AE601E70096
:101B3000088C012426F66F007A011726DEB70125EE
:101B40007F01197F011732F60125102A1B7D012420
:101B500027037E3BCFCE0124E600E701098C011963
:101B600026F67F011A4C20E30C44B700C007B701EA
:101B7000418606CE0124FF012ACE0000FF0128F68F
:101B800000C0C100270C6F054A274109FF01285AF0
:101B900020F0C601F501412715FE012AE60009FFE4
:101BA000012AFE0128E70509FF01284A271EFE0138
:101BB0002AE6005858585809EB0009FF012AFE018F
:101BC00028E705094A2705FF012820E27E6420BD99
:101BD00053567F00817E471F860297437E3C1D86B9
:101BE00001974397447E3C1D860397438680974424
:101BF0007E646586049743868197447E6465860586
:101C000097437F00447E6465860697437E646586BD
:101C10000797437E6465860897437E6465BD3932C5
:101C20009643810E24037E46FB39860E97437F013F
:101C30005C7E3932860F97437F015C7E3932861095
:101C400097437F015C7E39328603F6015C2605C628
:101C5000107E3AD8C6907F015C7E3AD87F0081BD65
:101C6000471FD69A2B2E9605270F810127037E53F7
:101C7000569604813124F7205296042717BD3CE97B
:101C80007F0005C690D79AD6048699108B011997C4
:101C9000047E3D169605F60816C501270981102B0E
:101CA0002A27147E53568101270424F7261D960403
:101CB000812124EF4F20089604812124E68609978C
:101CC00005BD3CDA860197057E3D16BD3CDA7F00F6
:101CD000057E3D167F0081BD471FD69A2B13D60582
:101CE000270BC10127037E5356C600201DC60120C5
:101CF00019D6052710B6081685012706C10925053E
:101D000027037E53564FBD4B965CD762BD5D7E392F
:101D10007F0081BD471FD69A2B16960526E4D60470
:101D2000C130270224DC8699108B3119164F201000
:101D300096052704810126CAD604CB301924014C0C
:101D4000BD4B96C19724BBD7637E5EB4BD3D56168E
:101D500026037E3FA639CE001FBD42DA270139DEB9
:101D60001FDF23DE21DF259626811822162B1796EA
:101D7000258160220E2B094F9124260791232603EB
:101D80007E3E1B7E3E22811222F62B149625813048
:101D900022EE2B5E4F912426E7912326E37E3DF22F
:101DA00081062B14224C9625816022462B0A7D0049
:101DB00024263F7D0023263A7F0017BD27C4260630
:101DC00096268102250FDE23DF0FDE25DF117E3F01
:101DD000A400002004CE3DD1DFC1CE0023DFC3CE5E
:101DE000000FDFC5860497C7BD4992868097177E8E
:101DF0003FA48601971796234624128601D6892789
:101E000009D68A2705BD3F812003BD3F65DE23DF5C
:101E10000FDE25DF11BD3F247E3FA4860297177E8B
:101E20003E678603971796234424128601D6892796
:101E300009D68A2705BD3F812003BD3F65DE23DF2C
:101E40000FDE25DF11BD3F24960F4424148602D6F1
:101E5000892709D68A2705BD3F8120CABD3F652055
:101E6000C5BD3F247E3FA47F0820962644444444B9
:101E7000B708219626840FB70821B60821840F974A
:101E800012962544444444B70821B60821165858F0
:101E900058589625840FB70821B60821840F1B9740
:101EA00011962444444444B70821B60821165858D2
:101EB00058589624840FB70821B60821840F1B9721
:101EC00010962344444444B70821B60821165858B4
:101ED00058589623840FB70821B60821840F1B9702
:101EE0000FB6082184F026037E3FA41654545454A0
:101EF0009689270B968A270717BD3F817E3FA486C8
:101F00000310BD3F654F4C9B0F19970F860099102A
:101F1000199710860099111997118600991219972F
:101F2000127E3FA4960F44850827028BFDD61054DD
:101F300024028B509706C5082702CBFD9611442436
:101F400002CB50D707850827028BFDD612542402F6
:101F50008B509708C5082702CBFDD709DE06DF0F97
:101F6000DE08DF11390C992319972386009924196B
:101F70009724860099251997258600992619972672
:101F800039B7009D7F009E7F009F7F00A0CE009DFF
:101F9000DFC3CE0023DFC1CE0023DFC5860497C791
:101FA000BD49AF394F39BD4334BD5F79BD591EBD01
:101FB000504BBD5E8996FB8A0297FBB60C0B84F7EB
:101FC000B70C0BBD27C4263EB6064484FEB70644B4
:101FD000D6172B22D118271EC40FCE4027BD4C3850
:101FE000B7062EDE25FF0631DE23FF062F8661C6EB
:101FF00005CE0632200D86707D00172A014CC604DE
:00000001FF
